:0A1CE10000010202030304040505DC
:100AEA00E4F55AF559F558F557C20AC207C209C2C0
:100AFA0008121C13120DED7E167F008E0A8F0B75DD
:100B0A00121675131275081675091C7510167511CB
:100B1A004A751416751578EE54E07003020C317597
:100B2A005B00755C808E5D8F5EC374A29FFF741636
:100B3A009ECF2402CF3400FEE48F568E55F554F52D
:100B4A0053F552F551F550F54FAF56AE55AD54AC7D
:100B5A0053AB52AA51A950A84FC312088F5026E589
:100B6A005C2552F582E55B3551F58374CDF0E5528B
:100B7A002401F552E43551F551E43550F550E43588
:100B8A004FF54F80C4E4F552F551F550F54FAF5685
:100B9A00AE55AD54AC53AB52AA51A950A84FC3128B
:100BAA00088F5031AE51AF52E55E2FF582E55D3EBA
:100BBA00F583E0FDE55C2FF582E55B3EF583EDF01C
:100BCA00EF2401F552E43EF551E43550F550E43591
:100BDA004FF54F80B9855B0A855C0B74002480FF52
:100BEA00741634FFFEC3E5139FF513E5129EF51242
:100BFA00C3E50D9FF50DE50C9EF50CC3E50F9FF5BA
:100C0A000FE50E9EF50EC3E5099FF509E5089EF569
:100C1A0008C3E5119FF511E5109EF510C3E5159F70
:100C2A00F515E5149EF514D2E843D82090E668E05D
:100C3A004409F090E65CE0443DF0D2AF90E680E0F3
:100C4A0020E105D20B1219A990E680E054F7F0537F
:100C5A008EF8C20A3008051208C6C208300A2912DC
:100C6A0012FE5024C20A121B5920071690E682E08F
:100C7A0030E704E020E1EF90E682E030E604E0208D
:0D0C8A00E0E4121A33121D761213B880C771
:1008C60090E6B9E070030209771470030209F42474
:1008D600FE7003020A7724FB700302097114700389
:1008E60002096B14607314607624056003020AD64D
:1008F600121D784003020AE290E6BBE024FE602265
:1009060014603324FD601114602224067048E50A41
:1009160090E6B3F0E50B8037E51290E6B3F0E51309
:10092600802DE50C90E6B3F0E50D8023E50E90E60C
:10093600B3F0E50F801990E6BAE0FF121A5FAA0637
:10094600A9077B01EA494B600DEE90E6B3F0EF9004
:10095600E6B4F0020AE2020ADB121CB0020AE21254
:100966001D33020AE21217F4020AE2121C9E020A60
:10097600E2121D7A4003020AE290E6B8E0247F60A4
:100986001514601924027063A207E43325E0FFA260
:1009960009E4334F8041E490E740F0803F90E6BCA5
:1009A600E0547EFF7E00E0D394807C0040047D010D
:1009B60080027D00EC4EFEED4F24E1F582741C3E74
:1009C600F583E493FF3395E0FEEF24A1FFEE34E6D2
:1009D6008F82F583E0540190E740F0E4A3F090E6BF
:1009E6008AF090E68B7402F0020AE2020ADB121D1C
:1009F6007C4003020AE290E6B8E024FE6016240278
:100A06006003020AE290E6BAE0B40105C207020AF0
:100A1600E2020ADB90E6BAE0705590E6BCE0547E4E
:100A2600FF7E00E0D394807C0040047D0180027D3F
:100A360000EC4EFEED4F24E1F582741C3EF583E496
:100A460093FF3395E0FEEF24A1FFEE34E68F82F5A7
:100A560083E054FEF090E6BCE05480131313541F59
:100A6600FFE0540F2F90E683F0E04420F0806D8085
:100A760064121D7E506690E6B8E024FE60192402DA
:100A8600705A90E6BAE0B40104D207804F90E6BAF5
:100A9600E064026047803E90E6BCE0547EFF7E0044
:100AA600E0D394807C0040047D0180027D00EC4E02
:100AB600FEED4F24E1F582741C3EF583E493FF338B
:100AC60095E0FEEF24A1FFEE34E68F82F5838008E1
:100AD600120080500790E6A0E04401F090E6A0E006
:030AE6004480F059
:010AE90022EA
:030033000215FCB7
:0415FC0053D8EF329F
:101C1300758CE0758AC0E58954F04401F589758EA9
:081C230003D28CD2A9D2AF223A
:03000B0002146973
:10146900C0E0C0F0C083C082C0D075D000C000C049
:1014790001C002C003C004C005C006C007758CE0E6
:10148900758AC0D28CE47F607EEAFDFCAB4EAA4D22
:10149900A94CA84BC312088F5019AF4EAE4DAD4C95
:1014A900AC4BEF2401F54EE43EF54DE43DF54CE43B
:1014B9003CF54BE47F01FEFDFCAB4EAA4DA94CA8BF
:1014C9004BC312088F7008E5A054F02534F5A0E548
:1014D9002B2401FFE4352AFEE4FCFDAB4EAA4DA9FD
:1014E9004CA84BC312088F700553A0F0C28CD007CB
:1014F900D006D005D004D003D002D001D000D0D07E
:09150900D082D083D0F0D0E03292
:1016000012010002000000401816234000000102F1
:1016100000010A06000200000040010009022E003D
:1016200001010080FA0904000004FF000000070522
:1016300001024000000705820200020007050202C5
:101640000002000705810240000009022E0001018E
:101650000080FA0904000004FF00000007050102F1
:101660004000000705820240000007050202000258
:101670000007058102400000040309041003510023
:10168000480059002D004300430044001603510058
:10169000480059002D0037002000200020002000C5
:0416A0002000000026
:10102000608028000205020202020207000000029E
:10103000000002000A2B0B13111511110000000013
:101040000000003F02050202020202070000000247
:10105000000002000A2B130B0915111100000000FB
:101060000000003F032A03030303030700000002FC
:10107000000002000A2B2B131115111100000000B3
:101080000000003F032A03030303030700000002DC
:10109000000002000A2B130B0915111100000000BB
:1010A0000000003F602428870000000000000000CE
:1010B0000000000000000000000000000000000030
:1010C00000000000000000000000000047288080B1
:0610D000000011CA4E00F1
:1011B60090E60174CAF090E6F574FFF0902880E09E
:1011C60090E6F3F0902881E090E6C3F0902882E064
:1011D60090E6C1F0902883E090E6C2F0902885E082
:1011E60090E6C0F0902886E090E6F4F075AF0774BC
:1011F60028F59A7400F59B759DE4E4F59EFF90E64C
:101206007BE090E67CF00FBF80F490E67174FFF00F
:10121600F5B490E672E04480F043B680000000E446
:1012260090E6C4F000000090E6C5F0902887E090B4
:10123600E6C6F0902888E090E6C7F0902889E0900E
:10124600E6C8F090288AE090E6C9F090288BE090F6
:10125600E6CAF090288CE090E6CBF090288DE090DE
:0B126600E6CCF090288EE090E6CDF082
:01127100225A
:03004300021300A5
:0300530002130095
:10130000021C2B00021C8800021C7200021C4300FD
:101310000218A50002183100021D8000021D810084
:10132000021D8200021D830002179C0002172D007F
:10133000021D8400021D8500021D8600021D87001B
:10134000021D8800021D8100021D8900021D8A0005
:10135000021D8B00021D8C00021D8D00021D8E00DF
:10136000021D8F00021D8100021D8100021D8100EF
:10137000021D9000021D9100021D9200021D9300AB
:10138000021D9400021D9500021D9600021D97008B
:10139000021D9800021D9900021D9A00021D9B006B
:1013A000021D9C00021D9D00021D9E00021D9F004B
:0813B000021DA000021DA100B6
:101A330090E682E030E004E020E60B90E682E030BE
:101A4300E119E030E71590E680E04401F07F147E71
:0C1A5300001215B690E680E054FEF02270
:101B590090E682E044C0F090E681F04387010000FE
:041B69000000002256
:1019A900300B0990E680E0440AF0800790E680E079
:1019B9004408F07FDC7E051215B690E65D74FFF0F1
:0F19C90090E65FF05391EF90E680E054F7F02244
:021A5F00A907D5
:101A6100AE14AF158F828E83A3E064037017AD01AE
:101A710019ED7001228F828E83E07C002FFDEC3EF8
:091A8100FEAF0580DF7E007F004E
:011A8A002239
:1015B6008E658F6690E600E054187012E566240189
:1015C600FFE43565C313F565EF13F566801590E600
:1015D60000E05418FFBF100BE56625E0F566E565EB
:1015E60033F565E5661566AE65700215654E6005F0
:0615F600121B6D80EE22C5
:101B6D007400F58690FDA57C05A3E582458370F98B
:011B7D002245
:1010D600C1820223000002311040C100C106C105D1
:0E10E600C104044700000000043A00000000AE
:081AB70090E679F07F057E0046
:101ABF008E658F66E566456560177F957E00121B04
:101ACF00AA000000000000E566156670E715658046
:021ADF00E32200
:100DED0090E600E054E74410F00000000000009091
:100DFD00E61074A0F000000090E60B7401F090E690
:100E0D001274E0F0000000E490E613F00000009092
:100E1D00E614F000000090E615F000000090E618D2
:100E2D00740CF000000090E6D27402F090E60474A9
:100E3D0080F00000007402F0000000E4F0000000FB
:100E4D001211B6E490E671F075B4FF90E672F0758C
:100E5D00B6BF75B1BF90E670F075B2FFC28CD28788
:100E6D00121D5375230275240000000090E61074C6
:100E7D00A0F000000000000090E611F000000090CE
:100E8D00E65EE04408F0000000E490E68DF090E6A8
:100E9D005EE04404F0000000E490E68FF0121A06C4
:100EAD00C2A1D2867F9A7E00121CEB75280075298F
:100EBD00B47542017543907531107532B87545069C
:100ECD0075462C121D4B90E67AE054FEF0E4FD7F42
:100EDD00901219457F647E001215B67DFF7F421278
:100EED0019457F647E001215B67D827F4E1219451D
:100EFD00121C5B7535FFE4F53890E782E535F0900F
:0B0F0D00E781E538F0121D6C021D5357
:1016A400E538D3940040037535FFD20590E678E021
:1016B4004480F07491121AB790E679E090E7C01272
:1016C4001ABA90E679E090E7C1121ABA90E679E086
:1016D40090E7C2121ABA90E679E090E7C3121ABAF8
:1016E40090E678E04440121ABA90E678E04480F03C
:1016F4007442121AB790E679E535121ABA90E67870
:10170400E04440121ABA90E678E04480F090E6791A
:10171400744E121ABA90E679E538121ABA90E6783D
:09172400E04440121ABAC2052289
:1013B800E54A2401F54AE43549F549E43548F54854
:1013C800E43547F547E47FE87E03FDFCAB4AAA49CC
:1013D800A948A847C312088F7006FD7F90121945C7
:1013E800E4FB7A08F9F8AF4AAE49AD48AC471207B2
:1013F800E7E4FB7A08F9F812075CC3E54A9FFFE5C2
:10140800499EFEE5489DFDE5479CFCE4FBFAF9F89A
:10141800C312088F7003121BF9E47F207E4EFDFC77
:10142800AB4AAA49A948A847C312088F7009121DD8
:10143800681216A4121D6CE47F407E9CFDFCAB4A2A
:10144800AA49A948A847D312088F400CE4F54AF5E1
:1014580049F548F547121BF9300105120C97C201EE
:011468002261
:0212FE00D322F9
:021D7600D32276
:021D7800D32274
:1017F40090E680E030E71800000090E6207402F0E4
:10180400000000E490E621F0000000D202801600FF
:101814000000E490E620F000000090E6217440F01F
:0D182400000000C20290E6BAE0F540D322B9
:101C9E0090E740E540F0E490E68AF090E68B04F0A1
:021CAE00D3223F
:081D330090E6BAE0F527D32287
:101CB00090E740E527F0E490E68AF090E68B04F0A8
:021CC000D3222D
:021D7A00D32272
:021D7C00D32270
:021D7E00D3226E
:10008000E4F55FF56090E6B9E01208A000B4B300B3
:10009000F9B50247B6027FC102FDC20348C503ACF1
:1000A000C603E1C90466CA049ACB0529CC0573CD01
:1000B00000000601E490E68AF090E68BF090E6A05E
:1000C000E020E1F990E68BE0F55FE4F5B5F5B3905B
:1000D000E60174CAF0E490E6C3F090E6C27411F051
:1000E000D20100000090E6047480F0000000740269
:1000F000F0000000E4F0020603E490E68AF090E6E7
:100100008BF090E6A0E020E1F990E68BE0F55FD37C
:10011000943F4024E4F56074402560F582E434E7C0
:10012000F583E0FF74AB2560F582E43428F583EFB6
:10013000F00560E560B440DF7F8A7E00121CEB9022
:1001400028ABE0FF7E00121CF49028ABE0FF7E009D
:10015000121CFD9028ABE0FF7E00121D069028AC1B
:10016000E075F004A4FFAEF0121D0F9028ACE0750E
:10017000F004A4FFAEF0121D189028ACE075F00456
:10018000A4FFAEF0121D219028B0E0C394025013DA
:100190009028CCE090E6C07005744EF08016749CF8
:1001A000F080119028CCE090E6C07005749FF0803C
:1001B00003749DF09028CEE0F5399028CBE0F53718
:1001C0009028CFE0F5419028D9E0F536A3E0FEA3D2
:1001D000E07C002400F526EC3EF5259028B1E0F502
:1001E00033E53370037533019028B6E0FEA3E07C5D
:1001F000002400F529EC3EF528A3E0FEA3E024004E
:10020000F543EC3EF5429028B2E0FEA3E02400F571
:1002100032EC3EF531A3E0FEA3E02400F546EC3ECF
:10022000F5459028BCE0FEA3E02400F53FEC3EF548
:100230003E9028BAE0FEA3E02400F530EC3EF52F16
:10024000E4FD7F900203DBE4F56074AB2560F5828A
:10025000E43428F583E0FF74402560F582E434E758
:10026000F583EFF00560E560B40ADF000000E4907C
:10027000E68AF000000090E68B740AF0020603E4C0
:1002800090E68AF090E68BF090E6A0E020E1F9900D
:10029000E68BE0F55FC298D394005003020603900A
:1002A000E740E0940A5007E02430FF121CD490E7A6
:1002B00040E0B40A057F61121CD490E740E0B40B23
:1002C000057F62121CD490E740E0B40C057F6312F6
:1002D0001CD490E740E0B40D057F64121CD490E775
:1002E00040E0B40E057F65121CD490E740E0640F37
:1002F00060030206037F66121CD402060390E740E7
:1003000074C9F0A37403F0A3740CF0A37426F0A3D3
:100310007407F0A374EEF0A37401F0A37403F0A3C8
:100320007453F0300205E4A3F0800690E74974FFAF
:10033000F0000000E490E68AF000000090E68B7484
:100340000AF0121A0602060390E678E04480F09064
:10035000E6797491F07F647E00121BAA90E679E042
:1003600090E740F07F647E00121BAA90E679E0904F
:10037000E741F07F647E00121BAA90E679E090E7E7
:1003800042F07F647E00121BAA90E679E090E7437A
:10039000F090E678E04440F0000000E490E68AF057
:1003A00000000090E68B7404F0020603E490E68AF5
:1003B000F090E68BF090E6A0E020E1F990E68BE08B
:1003C000F55FD39401500302060390E741E0FD7FFF
:1003D0004212194590E740E0FD7F4E121945020692
:1003E00003E490E68AF090E68BF090E6A0E020E14E
:1003F000F990E68BE0F55FD3940150030206039079
:10040000E740E05480C4131313540124FF92A3E087
:100410005440C41313540324FF92A2E05420C41385
:10042000540724FF92A1E05410C4540F24FF92A05B
:10043000A3E075F00AA4FFAEF01215B690E740E015
:100440005408131313541F24FF92A3E054041313EE
:10045000543F24FF92A2E05402C31324FF92A1E070
:100460001392A002060390E6BCE0756100F56220DD
:1004700005FDAD6290E6BEE0FB7EE77566E7756759
:10048000407FA0121B7EAD6290E6BEE0FB7EE7756A
:1004900066E77567407FA002055AE490E68AF0900F
:1004A000E68BF090E6A0E020E1F990E6BCE0D39482
:1004B0000750030206032005FD78EB7C287D017BB5
:1004C000017AE679BC7E007F011206D590E6BEE097
:1004D000FF7E0078EC7C287D017B017AE779401271
:1004E00006D590E6BEE004FD7A287BEB7F50121B18
:1004F000DD78EB7C287D017B017AE679BC7E007F8C
:10050000011206D590E6BEE0FF7E0078EC7C287DE7
:10051000017B017AE779401206D590E6BEE004FD42
:100520007A287BEB7F500205FC90E6BCE075610009
:10053000F5622005FDAD6290E6BEE0FB7EE77566E4
:10054000E77567407FA2121B7EAD6290E6BEE0FBBE
:100550007EE77566E77567407FA2121B7EE490E632
:100560008AF000000090E6BEE090E68BF00000000C
:10057000020603E490E68AF090E68BF090E6A0E0B5
:1005800020E1F990E6BCE0D3940740772005FD78A0
:10059000EB7C287D017B017AE679BC7E007F01122D
:1005A00006D590E6BEE0FF7E0078EC7C287D017BDE
:1005B000017AE779401206D590E6BEE004FD7A287C
:1005C0007BEB7F51121BDD78EB7C287D017B017A70
:1005D000E679BC7E007F011206D590E6BEE0FF7E84
:1005E0000078EC7C287D017B017AE779401206D502
:1005F00090E6BEE004FD7A287BEB7F51121BDD8084
:0406000002D322C33C
:0106040022D3
:101C2B00C0E0C083C082D2085391EF90E65D74018F
:081C3B00F0D082D083D0E0322A
:101C7200C0E0C083C0825391EF90E65D7404F0D05F
:061C820082D083D0E032A5
:101C8800C0E0C083C0825391EF90E65D7402F0D04B
:061C980082D083D0E0328F
:1018A500C0E0C083C08285100C85110D850D828531
:1018B5000C83A37402F085080E85090F850F8285B8
:1018C5000E83A37407F05391EF90E65D7410F0D08A
:0618D50082D083D0E03256
:101C4300C0E0C083C082D20A5391EF90E65D74086E
:081C5300F0D082D083D0E03212
:10183100C0E0C083C08290E680E030E72085080CDC
:1018410085090D850D82850C83A37402F085100E28
:1018510085110F850F82850E83A37407F05391EFD5
:0D18610090E65D7420F0D082D083D0E0329C
:011D80003230
:011D8100322F
:011D8200322E
:011D8300322D
:10179C00C0E0C0F0C083C082C0D075D000C000C013
:1017AC0001C002C003C004C005C006C007C2AF120E
:1017BC001D6800000090E68F7404F0000000539147
:1017CC00EF90E65FE04404F0121D6CD2AFD007D06E
:1017DC0006D005D004D003D002D001D000D0D0D098
:0817EC0082D083D0F0D0E0327E
:0D172D00C0E0C083C082C0D075D000C007EE
:10173A00C2AF90E6A1E020E1F990E780E0146012E0
:10174A002404601C14601D14602414702675220081
:10175A00802190E782E0F53590E781E0F538801343
:10176A00C28C800F90E781E024FF920680057522E3
:10177A0000D20300000090E68DE4F05391EF90E66A
:07178A005FE04408F0D2AF5C
:0B179100D007D0D0D082D083D0E0324F
:011D8400322C
:011D8500322B
:011D8600322A
:011D87003229
:011D88003228
:011D89003227
:011D8A003226
:011D8B003225
:011D8C003224
:011D8D003223
:011D8E003222
:011D8F003221
:011D90003220
:011D9100321F
:011D9200321E
:011D9300321D
:011D9400321C
:011D9500321B
:011D9600321A
:011D97003219
:011D98003218
:011D99003217
:011D9A003216
:011D9B003215
:011D9C003214
:011D9D003213
:011D9E003212
:011D9F003211
:011DA0003210
:011DA100320F
:061512008F638C648D65FF
:1015180053630753A0BF121BA6E4F566F567C374AF
:10152800029567FFE563A807088002C313D8FC305B
:10153800E00543A020800353A0DF121BA6121BA3C3
:1015480053A0EF121BA60567E56770020566C394F2
:1015580003E5666480948040C5E4F566F567C37466
:10156800099567FFE565AE64A807088005CEC31333
:10157800CE13D8F930E00543A020800353A0DF1232
:101588001BA6121BA353A0EF121BA60567E56770E5
:10159800020566C3940AE5666480948040C043A04F
:0E15A80040121BA653A0BF7F0A7E00021BAAA2
:091CEB00AD07AC06E4FF0215127E
:091CF400AD07AC067F04021512D5
:091CFD00AD07AC067F05021512CB
:091D0600AD07AC067F06021512C0
:091D0F00AD07AC067F01021512BC
:091D1800AD07AC067F02021512B2
:091D2100AD07AC067F03021512A8
:101945008D63AD0790E678E04480F090E679EDF0A0
:101955007F647E00121BAA90E679E563F07F647EC2
:1019650000121BAA90E678E04440F07F647E0002F6
:021975001BAAAB
:071BA30043A0107F0A7E0041
:101BAA00EF7803C333CE33CED8F9FFEF4E6007EF99
:071BBA001F70F81E80F522E8
:031D7000C282220A
:031D7300D28222F7
:051D5900C280D28122CE
:051D5E00D280D28122B9
:051D6300C280C28122D4
:061D5300121D70021D5E6E
:101BF900121D59121D737F017E00121BAA121D703E
:0A1C0900121D5E7F017E00021BAA7F
:101CC200E4FDFC121BF90DBD00010CBC1DF5BD4C61
:011CD200F21F
:011CD30022EE
:1019D800121D597F057E00121BAA121D63121D736A
:1019E8007F057E00121BAA121D59121D707F057EED
:0E19F80000121BAA121D5E7F057E00021BAAB4
:081D3B00C286121BA6D286220B
:101A0600E4F563F56443B1807F1E7E001215B6537C
:101A1600B17F7F1E7E001215B60564E5647002056F
:0C1A260063C39405E5636480948040D99C
:011A32002291
:041D680043B18022E1
:041D6C0053B17F22CE
:091D2A007F4F121CD443B12022AA
:081D430053B1DF7F43021CD401
:1010F500E4FFFEE53BFDE4FCFB7A01F9F81207E7A6
:10110500E4FB7A01F9F81207E78F2CE4FFE53CFED2
:10111500E4FDFCFB7A01F9F81207E78F2EE53DFFA8
:101125008F2DE537B40102C287121D2AE539706D8E
:10113500752201E52C75F040A485F063F564AF22B6
:101145007E00AC63AD6412074AD3EF9400EE9400C1
:1011550040147FC47E03121ABF1216A4E5641564F9
:1011650070DC156380D8756300852E64AF227E0020
:10117500AC63AD6412074AD3EF9400EE94004014BB
:101185007FC47E00121ABF1216A4E564156470DCD4
:10119500156380D8AF2D7E001215B6800975220122
:1011A500E522640160FA121D43E537B40102D287D6
:0111B5002217
:101A8B00AD07AC06D3ED9400EC9400401E000000B3
:101A9B00EE90E6D0F0000000ED90E6D1F0000000F3
:0C1AAB0075BB04000000E5BB30E7FB2227
:08186E008C638D64AB07AA0630
:10187600E4FDFCC3ED9564EC95635022EA90E6D056
:10188600F0000000EB90E6D1F000000075BB06000A
:0E1896000000E5BB30E7FB0DBD00010C80D566
:0118A4002221
:101AE100AD07AC06000000ED25E0EC3390E6D0F048
:101AF100000000ED25E090E6D1F000000075BB0488
:091B0100000000E5BB30E7FB2207
:100C9700C2A3121D6CC2039028AEE0FFE4FCFDFE68
:100CA700FB7A01F9F812075CC004C005C006C0074B
:100CB7009028ADE0FFE4FCFDFEFBFA7901F812078E
:100CC7005CD003D002D001D000EF2BFBEE3AFAED57
:100CD70039F9EC38F89028AFE0FFE4FCFDFEEB2F84
:100CE700F53DEE3AF53CED39F53BEC38F53AE47F66
:100CF70091AB3DAA3CA93BA83AD312088F4029E5FE
:100D07003D246FF53DE53C34FFF53CE53B34FFF50D
:100D17003BE53A34FFF53A121D3B1210F5E5304535
:100D27002F7014121CC2800FE530452F7003121C60
:100D3700C2121D3B1210F51219D8121D6830030399
:100D4700020DECE4F561F562C3E5629529E561956D
:100D570028500D121BF90562E56270EC056180E809
:100D6700E536D39400400CE536FD7C00AF32AE315A
:100D770012186ED3E5269400E52594004007AF26A8
:100D8700AE25121AE1E4F55FF560C3E5609546E527
:100D97005F9545502C121B0AE4F561F562C3E562C5
:100DA70095337480F8656198500D121BF90562E55B
:100DB7006270EA056180E60560E56070CD055F80D9
:100DC700C9E4F561F562C3E5629543E56195425073
:100DD7000D121BF90562E56270EC056180E8AF3F13
:050DE700AE3E121A8B64
:010DEC0022E4
:101B0A00000000E53225E0E5313390E6D0F0000030
:101B1A0000E53225E090E6D1F000000075BB040034
:081B2A000000E5BB30E7FB22DF
:101C5B00E490E608F075C83443985053877FC2ACC4
:071C6B0075CBFF75CA64226E
:0D1CD400309902C2998F993099FDC2992272
:101B320090000020981CA3AF82AE83E4FCFD7BFAE8
:101B42007AFFF9F8C31208795004D2008004C20067
:061B520080E1C298AF998A
:011B5800226A
:041B7E008F638B6581
:101B820090290BEDF0E563C313FF7A297B0B7D01EE
:101B9200121BDDE563C313FFAB67AA66AD65021BCB
:011BA200C181
:081D4B00E4F51BD2E9D2AF223E
:1018DB0090E678E020E6F9C2E990E678E04480F003
:1018EB00EF25E090E679F090E678E030E0F990E6CD
:1018FB0078E04440F090E678E020E6F990E678E076
:06190B0030E1D6D2E92212
:10197700A90790E678E020E6F9E51B702390E67862
:10198700E04480F0E925E090E679F08D16AF03A9F1
:10199700077517018A188919E4F51A751B01D322EF
:0219A700C32259
:10191100A90790E678E020E6F9E51B702590E678C6
:10192100E04480F0E925E0440190E679F08D16AFBE
:1019310003A9077517018A188919E4F51A751B039C
:04194100D322C322C8
:03004B00020F1889
:100F1800C0E0C083C082C085C084C086758600C01A
:100F2800D075D000C000C001C002C003C006C00711
:100F380090E678E030E206751B0602100290E6782B
:100F4800E020E10CE51B64026006751B0702100235
:100F5800E51B24FE605F14603624FE7003020FF365
:100F680024FC7003020FFF24086003021002AB1771
:100F7800AA18A919AF1A051A8F827583001206FBE1
:100F880090E679F0E51A65167070751B05806B9010
:100F9800E679E0AB17AA18A919AE1A8E82758300F4
:100FA800120728751B02E5166401704E90E678E07A
:100FB8004420F08045E51624FEB51A0790E678E04F
:100FC8004420F0E51614B51A0A90E678E04440F09B
:100FD800751B0090E679E0AB17AA18A919AE1A8E0E
:100FE80082758300120728051A800F90E678E0447E
:100FF80040F0751B008003751B005391DFD007D0AC
:1010080006D003D002D001D000D0D0D086D084D072
:0810180085D082D083D0E032C4
:101BC100121911E51B24FA600E146006240770F344
:0C1BD100D322E4F51BD322E4F51BD32241
:101BDD00121977E51B24FA600E146006240770F3C2
:0C1BED00D322E4F51BD322E4F51BD32225
:0300000002127277
:0C127200787FE4F6D8FD7581670212B9A0
:10060500E709F608DFFA8046E709F208DFFA803ED7
:1006150088828C83E709F0A3DFFA8032E309F608C4
:10062500DFFA8078E309F208DFFA807088828C832C
:10063500E309F0A3DFFA806489828A83E0A3F608E0
:10064500DFFA805889828A83E0A3F208DFFA804CBA
:1006550080D280FA80C680D4806980F28033801091
:1006650080A680EA809A80A880DA80E280CA8033FA
:1006750089828A83ECFAE493A3C8C582C8CCC58372
:10068500CCF0A3C8C582C8CCC583CCDFE9DEE78042
:100695000D89828A83E493A3F608DFF9ECFAA9F0C1
:1006A500EDFB2289828A83ECFAE0A3C8C582C8CC17
:1006B500C583CCF0A3C8C582C8CCC583CCDFEADE30
:1006C500E880DB89828A83E493A3F208DFF980CC92
:1006D50088F0EF60010E4E60C388F0ED2402B4048B
:1006E5000050B9F582EB2402B4040050AF23234532
:0606F500822390065573FC
:1006FB00BB010CE58229F582E5833AF583E02250B4
:10070B0006E92582F8E622BBFE06E92582F8E222FD
:0D071B00E58229F582E5833AF583E4932217
:10072800F8BB010DE58229F582E5833AF583E8F007
:10073800225006E92582C8F622BBFE05E92582C8B3
:02074800F2229B
:10074A00EF8DF0A4A8F0CF8CF0A428CE8DF0A42EC3
:02075A00FE227D
:10075C00E88FF0A4CC8BF0A42CFCE98EF0A42CFC3C
:10076C008AF0EDA42CFCEA8EF0A4CDA8F08BF0A4BA
:10077C002DCC3825F0FDE98FF0A42CCD35F0FCEB19
:10078C008EF0A4FEA9F0EB8FF0A4CFC5F02ECD39DE
:0F079C00FEE43CFCEAA42DCE35F0FDE43CFC224B
:1007AB0075F008758200EF2FFFEE33FECD33CDCC05
:1007BB0033CCC58233C5829BED9AEC99E582984088
:1007CB000CF582EE9BFEED9AFDEC99FC0FD5F0D665
:1007DB00E4CEFBE4CDFAE4CCF9A88222B800C1B98F
:1007EB000059BA002DEC8BF084CFCECDFCE5F0CBCD
:1007FB00F97818EF2FFFEE33FEED33FDEC33FCEB06
:10080B0033FB10D703994004EB99FB0FD8E5E4F9C0
:10081B00FA227818EF2FFFEE33FEED33FDEC33FCAD
:10082B00C933C910D7059BE99A4007EC9BFCE99AA1
:10083B00F90FD8E0E4C9FAE4CCFB2275F010EF2FE6
:10084B00FFEE33FEED33FDCC33CCC833C810D707E6
:10085B009BEC9AE899400AED9BFDEC9AFCE899F821
:0E086B000FD5F0DAE4CDFBE4CCFAE4C8F922B4
:10087900EB9FF5F0EA9E42F0E99D42F0EC6480C8F6
:0608890064809845F02296
:10088F00EB9FF5F0EA9E42F0E99D42F0E89C45F0BF
:01089F002236
:1008A000D083D082F8E4937012740193700DA3A3E7
:1008B00093F8740193F5828883E4737402936860FB
:0608C000EFA3A3A380DFFB
:10127E00020AEAE493A3F8E493A34003F68001F292
:10128E0008DFF48029E493A3F85407240CC8C33371
:10129E00C4540F4420C8834004F456800146F6DF40
:1012AE00E4800B0102040810204080901020E47EA0
:1012BE00019360BCA3FF543F30E509541FFEE49335
:1012CE00A360010ECF54C025E060A840B8E493A3FC
:1012DE00FAE493A3F8E493A3C8C582C8CAC583CA27
:1012EE00F0A3C8C582C8CAC583CADFE9DEE780BEDF
:0110F40000FB
:00000001FF
